:030000000219FDE5
:03000B000200A848
:03002B000201547B
:03005B000202DDC1
:030073000202CABC
:1000800002030406080C10182030406080040608A3
:100090000C10182030406080A0C00003070F1F051F
:1000A000050D050205030302C2AFC0D0C0E0206207
:1000B00014E5256009E473E525F4F58AD262D0E001
:1000C000D0D0D2AF3285268AC262E526F46029D02C
:1000D000E0D0D0C293C295C297D2AF32C293C2953C
:1000E000C297206F0C206609740ED5E0FDE57B42B7
:1000F00090D0E0D0D0D2AF32758A00C28DD26201EA
:10010000F101B7306805206602D29301B730680567
:10011000206602D29501B7306805206602D29701A9
:10012000B7C29230680A206607740CD5E0FDD293FE
:1001300001B7C29430680A206607740CD5E0FDD27E
:100140009501B7C29630680A206607740CD5E0FDA9
:10015000D29701B7C2AFC2AD53E6EFC0D0C0E0D274
:10016000D3D2AFC2CEE52A6007207449152A21B543
:100170007800790020742EE580307E01F430E302AF
:1001800078FF53DACF207E0343DA20307E0343DA50
:1001900010C2D8C271E580307E01F430E30279FFED
:1001A000C3E89970CB306103752A18207403752A4F
:1001B00018885CD27020740DE52B6004152B21C5C6
:1001C00043DA01C2D82070024138A85C206102C223
:1001D00070207431C3E894F0400374F0F8E8C4541C
:1001E0000F28F87984B703024105C313C31387218D
:1001F000200802C313200A06C3C898F8410528F84E
:10020000500374FFF8C3E895655003E565F888224C
:10021000E52D54066022206B1FE536C333C333F847
:10022000E564C313C313F9C3952240028922E8256C
:1002300022F52250037522FF852224A824C3E52439
:1002400095614002A8618825E5667002417CC3E89B
:10025000AA669A5003E8FAE4F9EAC333FBE568F4C6
:100260005B29400D2567F8E56760021567400B4183
:100270007C0AC3E5679A5002056778FF8826C3E5C4
:100280002594404002D26420CF0AD0E0D0D043E68B
:1002900010D2AD32C2CF053A7801E52A600530743C
:1002A00002152AC3E55C94014005755F0041C075E5
:1002B0006000756900E55F2401F55F5003755FFF1D
:1002C000D0E0D0D043E610D2AD32C2AF53E67F7556
:1002D00092FA7593FFC260759104D2AF32C2AF53E8
:1002E000E6EFC2ADC0D0C0E0C0F0D2D3D2AFA8FB21
:1002F000A9FCC2D8307102614453DACF207E034397
:10030000DA10307E0343DA20D271E580307E01F4CA
:1003100020E302611B88278928A17153DACF207E50
:100320000343DA20307E0343DA10C2D8C27130743E
:1003300002A15D7800E580307E01F430E302A15D2A
:10034000885CA14553DACF207E0343DA20307E0358
:1003500043DA10C271206102811D53DACF207E037F
:1003600043DA10307E0343DA20C2D8D2718857892D
:1003700058C3E89555F8E99556F97B007E087A0050
:10038000C3E8948CE994005005755B00810F8821C7
:1003900078A2E6A8216055C3E894C8E99400500803
:1003A000E4D2E4FB7A0A61EAC3E89468E994015074
:1003B00008E4D2E3FB7A0F61EAC3E894D0E994023F
:1003C0005008E4D2E2FB7A1E61EAC3E894A0E99403
:1003D000055008E4D2E1FB7A3C61EAC3E89498E96D
:1003E00094085008E4D2E0FB7A787E00C3E895597F
:1003F000FCE9955AFD30E70AECF42401FCEDF434F5
:1004000000FD755B00C3EC9AED9E5003755B01889F
:1004100059895A8557558558567802A145C3E8959C
:1004200027F8E99528F9307C02A129307B02A1291F
:10043000307A02A1222075028140E9FDE8FC815F4B
:10044000E9C313F9E813F8307902A122E9C313F9DB
:10045000E813F8307802A122E9C313FDE813FC2069
:10046000612CC3EC941CED940240028176ED701E69
:0F047000C3EC94C850180529E52970021529C35B
:10047F00E529940A5002A15D755C00D270A15DE57B
:10048F0029600215297888E6F97400207F0878968C
:10049F00B90302789EE624FAFEE43400FFC3EC9E13
:1004AF00FCED9FFD9208B90310A2085007207609B2
:1004BF00D27681C8307602C276A2085016B9030DE3
:1004CF00ECF42401FCEDF43400FD0204E278007931
:1004DF0000A129B90315EC33FCED33FDC3EC940AED
:1004EF00FCED9400FD50047C007D00C3EC94FFED07
:1004FF009400400678FF7900A129EC8572F0A4C51D
:10050F00F0A2F733F87900400302054578FF790030
:10051F00020545E9C313F9E813F8307C0EE96002D0
:10052F0078FFC3E81338F8E43400F9C3E894FFE91F
:10053F009400400278FF885CD270206102A15D7444
:10054F001FF4552F4BF52FC274EB7002D274752A1E
:10055F0018307403752A0A306102A1712074035395
:10056F00DAFE207403752B06D0F0D0E0D0D0D2ADD8
:10057F0043E6103279010205A179030205A1790A38
:10058F000205A1791E0205A179640205A179C802AD
:10059F0005A17817E4D5E0FDD8FAD9F6227A147BB5
:1005AF00780205C87A107B8C0205C87A0D7BB402DD
:1005BF0005C87A0B7BC80205C87902E4C294D5E05E
:1005CF00FDD295D5E0FDC295D5E0FDD294D5E0FDE5
:1005DF00E920E002D29330E002D297E573D5E0FD37
:1005EF00E920E002C29330E002C2977496D5E0FD95
:1005FF00D9C9EAF8D5E0FDD8FBDBBEC29422C37C93
:10060F00007D0075F00005F0EA33FAEB33FB50F68E
:10061F00EB13FBEA13FAC3E9FFE8FEE89AF8E99B4C
:10062F00F95004EFF9EEF8B3EC33FCED33FDD5F0F0
:10063F00DFEDF9ECF822E889F08A20D2D4F8A9F09E
:10064F007B0030F70B7BFFF42401F8E9F43400F959
:10065F00E88520F0A4ADF0F8E98520F0A4AFF0FE16
:10066F00ED2EF974003FFA7C04C3EA13FAE913F98B
:10067F00E813F8DCF48BF030F70AE8F42401F8E91A
:10068F00F43400F9E889F0C2D4F8A9F02222C3E5C6
:10069F004113F9E54013F8C3E54498F8E54599F996
:1006AF00500CC3E89480E994FF40160206D4C3E8C7
:1006BF00947FE9940050030206D4787F79000206F4
:1006CF00D4788079FF8849894A22E5492546F8E59B
:1006DF004A3547F9854A20E4300701F43548FA30A6
:1006EF00E709C3EA94F04015020712C3EA940F50CA
:1006FF000302071278FF79FF7A0F02071278007949
:10070F00007AF0C3E5249561500AC3740195245013
:10071F000B020730E54A20E70E020730E54A30E7C3
:10072F0006884689478A482278A5E6FAC3E5493301
:10073F00F8E54A33F9D145E930E70BC3E89480E98E
:10074F0094FF4013E16AC3E8947FE994005002E1FB
:10075F006A787F7900E16A788079FFE820E715C32E
:10076F00E52398F84009C3E8940140030207917804
:10077F0001020791E8F424012523F84003020791B1
:10078F0078FF884B2278A6E6FAA847A948D145E911
:10079F0030E70CC3E89401E994FF40160207C5C384
:1007AF00E894FFE9940050030207C578FF7900022F
:1007BF0007C5780179FFE920E715C3E54B98F840A5
:1007CF0009C3E8940140030207EC78010207ECE843
:1007DF00F42401254BF840030207EC78FF8824220C
:1007EF0078FFC26420693D206A12D264C3E5419448
:1007FF000A4009C3E52594405002C26479A1E7601D
:10080F0023E541601F74FF8541F0848539F0306A1C
:10081F000375F005A4F8C5F0600278FFC3E895648E
:10082F005002A864886322C3E5409440E5419401D7
:10083F00E5635003140147046002F5632202084F79
:10084F002275E890227883E6FFE5E820ECF7A8BD53
:10085F00A9BE0570C3E57094084052757000E9FA9F
:0F086F0079A0E76044EA7007E571601B02088A10
:10087E00C3E895716010E5715006600C140208967D
:10088E000460F9020896E571F571C394A8401B75D2
:10089E0061C0C394054013756180C39405400B7508
:1008AE006140C39405400375610075BB0122E5618B
:1008BE00F460020561E570B4070375BB1E22743245
:1008CE0079A787F0A4C5F0A2F733F8C3E895614085
:1008DE0002A861882288248825882688642275408B
:1008EE00007541F022C2AF75C820A8CCA9CDAA3A96
:1008FE0030CF010A75C824D2AFAB3BAC3C883B89E4
:10090E003CC3E89BF8E99C206908F930670221FF97
:10091E00215CAD3D8A3DF9EA9DFA600478FF79FFCE
:10092E00AE3EAF3F8B3E8C3FA83BA93CC3E89EF842
:10093E00E99FF9C3E54113FBE54013FAE82AF540B8
:10094E00E93BF54150067540FF7541FF21A6AA40CF
:10095E00AB41AC40AD417E047F02C3EB9404400238
:10096E001E1FC3EB940840021E1FC3ED13FDEC13B4
:10097E00FCDEF7C3EA9CFAEB9DFBEF6009C3E913BB
:10098E00F9E813F8DFF7EA28FAEB39FB8A408B41D6
:10099E0050067BFF8B408B41C3EB94025002D26713
:1009AE003069047F0321D17892E6FFC3E537948244
:1009BE0040110FC3E53794A040010FC3EF940640DA
:1009CE00027F057E02E541C4540FF9E541C454F09F
:1009DE00F8E540C4540F28F8C3E89EFAE99400FBEA
:1009EE004009C3EA9402EB940050047A02E4FB41FE
:1009FE004BAA40AB41EBC4FEEAC4540F4EFCC3EA13
:100A0E009CFAEB9400FBC3E813C313F8EA28FAEB45
:100A1E003400FB8A408B41C3EB94024002C26778DC
:100A2E0002EBC4FE7B00EAC4540F4EFAC3EA98FAF6
:100A3E004005C3940250027A027892E6FF306002BB
:100A4E00414B855192855293D26043E680C3E49A1E
:100A5E00F8E49BF930670241D7E8FAE9FBD3E913D2
:100A6E00FDE813FC88518952C3EF94036038EF20E0
:100A7E00E00DE82CF8E93DF9ECFAEDFB020AA0E8EE
:100A8E0028F8E939F9C3E82402F8E93400F97AFEC6
:100A9E007BFFC3EF9403400E8A538B54884D894ECF
:100AAE008C4F8D50610B885389548A4D8B4E8C4FD1
:100ABE008D503069127553F07554FF754FF07550A7
:100ACE00FF7551F07552FF610BE8FAD3E813FC88FD
:100ADE0051C3EF94036020EF20E007E82CF8ECFA06
:100AEE0041F7E8282402F87AFEC3EF940340088AFF
:100AFE0053884D8C4F610B88538A4D8C4FE568C3DC
:100B0E00335002646BF5683060026115753402D2A1
:100B1E006043E680E52D54066034A840A941C3E940
:100B2E0013F9E813F8C3E913F9E813F8306904E987
:100B3E002440F9C2AF53E67F759100C3E498F59453
:100B4E00E499F595759104D26043E680D2AF22D236
:100B5E0065754300752000306C03752040020B7CD8
:100B6E00D265754300752040306C03752000780106
:100B7E007901206720E52D54066002C2657914E5DF
:100B8E0041C313700104F8C3941440027814306901
:100B9E0004781B791B206010E543600C306903D587
:100BAE003404D26D8127711D0543E59E7005E59BCA
:100BBE00020BC3E59A5440B5200281113069090831
:100BCE00C3E89940011861A320650A08C3E899405B
:100BDE0002617C61A3C265C2AF53E67F759100309E
:100BEE0067127594007595FE759104D26043E68088
:100BFE00D2AF617CAE40AF41C3E49EF594E49FF565
:100C0E009561F6C3E53394015002617C3065026153
:100C1E007CD802812561A3C26DC2AF53E67F759168
:100C2E0000855394855495759104854D92854E9308
:100C3E00D26043E680D2AFE52D54066008206A02EA
:100C4E000533020C63306D0D206C0A20650715818B
:100C5E001581021524227800306405306502780172
:0F0C6E00E53775F007A4F9E5F028F5F0E9A2F0F5
:100C7D0013A2F113A2F213F537C39478500375370D
:100C8D0078C3E53795384008D266C293C295C297AE
:100C9D00306002819D854F92855093D26043E680EE
:100CAD0022207D19C2AF754202C294D292306202E7
:100CBD00D297D2AF759F33759E00020EAFC2AF753E
:100CCD004202C294D296306202D293D2AF759F3354
:100CDD00759E00020EAF307243207D20C2AF75426B
:100CED0003900132757B10C297C296306204D29583
:100CFD00A101D294D2AF759E23020EAFC2AF754241
:100D0D0003900132757B10C293C292306204D2956A
:100D1D00A121D294D2AF759E22020EAF207D17C2B3
:100D2D00AF75420390010DC297306202D295D2AFDA
:100D3D00759E23020EAFC2AF75420390010DC29393
:100D4D00306202D295D2AF759E22020EAF207D1673
:100D5D00C2AF754204C292D296306202D295D2AF22
:100D6D00759E22020EAFC2AF754204C296D292306A
:100D7D006202D295D2AF759E23020EAF307249201A
:100D8D007D23C2AF754205900121757B04C295C2CA
:100D9D0094306204D293A1A7D292D2AF759F3375CE
:100DAD009E00020EAFC2AF754205900143757B40A8
:100DBD00C295C294306204D297A1CAD296D2AF75B1
:100DCD009F33759E00020EAF207D1AC2AF7542058E
:100DDD00900103C295306202D293D2AF759F3375E5
:100DED009E00020EAFC2AF754205900117C295303D
:100DFD0062E8D297D2AF759F33759E00020EAF2079
:100E0D007D16C2AF754206C296D294306202D2935D
:100E1D00D2AF759E23020EAFC2AF754206C292D2FB
:100E2D0094306202D297D2AF759E22020EAF30720D
:100E3D0043207D20C2AF754201900143757B40C2B6
:100E4D0093C292306204D297C159D296D2AF759E99
:100E5D0022020EAFC2AF754201900121757B04C213
:100E6D0097C296306204D293C179D292D2AF759E59
:100E7D0023020EAF207D17C2AF754201900117C23C
:100E8D0093306202D297D2AF759E22020EAFC2AFDF
:100E9D00754201900103C297306202D293D2AF75B1
:100EAD009E23C26622900101757B00C293C295C23A
:100EBD0097C292C294C296C26222788076FF08765B
:100ECD00FF0876FF0876FF08760308760408760794
:100EDD00087601087601087601788C76010876FF90
:100EED000876FF0876FF0876FF0876FF0876030878
:100EFD0076FF0876FF0876FF0876250876D0087607
:100F0D00FA0876FA0876040876FF08760108760066
:100F1D0008767A0876FF08760108760108760008CB
:100F2D007603087600227887E6FFC2727888E6C3DA
:100F3D0094036008C27DE630E102D27DC27E7889DD
:100F4D00E630E102D27EC3EF94026008758E01D2C5
:100F5D0073020F66758E00C273227880E6149000BE
:100F6D00809378A5F67881E6149000809378A6F6A4
:100F7D007886E61490008D9378A7F67886E6F53995
:100F8D00C394025003753902789CE67538FFB4029C
:100F9D00037538A0B4030375388278A3E614900066
:100FAD009A93F566D1B222227896E6FA7897E6FB07
:100FBD007888E6B40305C3EB940EFB307F047A000A
:100FCD007BFFC3EB9AFCC3948250027C8275720046
:100FDD000572EC8572F0A4C3E5F0947D40F222D247
:100FED007FF1B51205927A007B007C10120588E521
:100FFD005C2AFA74003BFBDCF37C04C3EB13FBEAC5
:10100D0013FADCF7FEC27F120FB522E5EF20E603DF
:10101D007520000520903DFFE520146006901FFF10
:10102D001460009304600375EF1253D9BF7581C02E
:10103D0043FF8012058375EF0243B203E5B324022B
:10104D0020E70DF521E5B120E0068521B343B1017F
:10105D00120EB27580FF75A40075F1FE75D4F7758B
:0E106D00900275A5FC75F2FC75D50075A0FD0E
:10107B0075A60275F30275D60075B0FF75A70175DD
:10108B00F4FF75E241120EB2E4F8F6D8FD75680173
:10109B00120EC712157578988673753001C2AF1290
:1010AB00059C1205AC1205921205B312059212059E
:1010BB00BA12059212168E12059C12059C120597F8
:1010CB00C2AF78FA79FA308307D9FBD8F7021C0044
:1010DB00120F33120F67120FB4120FB57898867375
:1010EB00120EB275881075890275C8247591047536
:1010FB00D84075A82275B80275E690759B80759DD2
:10110B0000759A80759C0075D10E75BC5875BB0126
:10111B0075BA1F75E880120583D2AF12084C75366D
:10112B000053DACF207E0343DA20307E0343DA10FC
:10113B0043DA01C2D8C27112059CD2617B037A0CCF
:10114B00E55B70077A0CDB030210CB120592207063
:10115B00030210CBC270E55CC3940240E1E52F544F
:10116B001F855E5DF55EB55DD5DAD5C26153DACF0D
:10117B00207E0343DA20307E0343DA10C2D8C271DB
:10118B0078A2E67008D274E52F54E0F52FC275757E
:10119B002900120597307409C3E529940A4002D23D
:1011AB007512058878023074027800C3E55C9840AC
:1011BB00F0C2AF1205AC1205AC1205ACD2AF1205E2
:1011CB009C754C007888E6B4030241B4120588780C
:1011DB008CE6C3940150030212B4E530C394015062
:1011EB00030212B4207435C3E55C94FF5003021262
:1011FB00B4C2AF1205C1D2AF120597C3E55C94011F
:10120B0050EFC2AF1205AC12058D1205ACD2AF1266
:10121B000597C3E55C94FF40E90217137F05D27F66
:10122B00120FB5120597C2AFC27F120FB5AE5CC3DA
:10123B00E55C947FD2AF407B120583C2AF1205C130
:10124B00D2AFDFDA120FECC3EE94057897F61205E6
:10125B009C1215B71216967F0AD27F120FB5120584
:10126B0097C2AFC27F120FB5AE5CC3E55C947FD261
:10127B00AF50E4120583C2AF1205AC12058D1205F7
:10128B00ACD2AFDFD4120FECEE24037896F6120536
:10129B009C1215B71216C5120597120FB5C3E55C54
:1012AB0094FF500221EF021713C3E55C954C4003EA
:1012BB00855C4C12059778017988E7B403027805B1
:1012CB00C3E55C98400221CFC2AF1205C11205C124
:1012DB001205C1D2AF12059C753000E4F531F53221
:1012EB000531E531F4703F0532789AE678191460D0
:1012FB0012783214600D787D14600878FA1460034C
:10130B00753200C3E53298401D120EB212058315DB
:10131B003275310078998673C2AF1205C1D2AF789E
:10132B0098867312059712058DE52A7005307402A5
:10133B0001CB78012074027806C3E55C9840A17854
:10134B0088E6C394036003120597E52A7003021025
:10135B00CBC2AF120EB2E4F522F523F524F525F539
:10136B0026F567D2AF7885E6C333F565E4F544F52A
:10137B0045F546F547F548F570F52CF52DF5377520
:10138B00700875BB1E120583120850E5E820ECFBB4
:10139B00A8BDA9BEE97001F88871120854757008D0
:1013AB0075BB1E120F33C2AF7561FF1208CC8522BD
:1013BB0061852262852263D2AF7522017524017586
:1013CB002501752601856069756A017888E6B40385
:1013DB0007C27D307602D27DD268D2697533001296
:1013EB000E0C120E3B1208EC1208F31208EC12084A
:1013FB00F31208EC120B6E12069C120C64120CAE5C
:10140B001208F3120B5D306E0312069D2067031258
:10141B0007EF306703120836120C64120CE3120844
:10142B00F3120B6E306E031206D9120C64120D5AA6
:10143B001208F3120B5D306E03120737120C641295
:10144B000D891208F3120B6E306E03120794120CF7
:10145B0064120E0C1208F3120850120B5D120C647E
:0F146B00120E3B1208541208F330692F8564618A
:10147A00856462856069756A0179187A0CC3E533F7
:10148A0099400CC269D26A8A357561FF0214A6C3F3
:10149A00E55C940140030213FF02152C306A1D20FB
:1014AA006C1AE535147006C26AD26B61FFF535C352
:1014BA00E55C940140030213FF02152C753600788F
:1014CA008279A4E760027803C3E55F9850543074C8
:1014DA0004E52A604D7888E6B40317207D05207656
:1014EA000781FC30760281FC206C07D26C8564612E
:1014FA00813E78F0306C058564617820C3E54198B7
:10150A00500261FF306C1BC26CC27D307602D27D04
:10151A00D26A75351285646161FF0536E55C600241
:10152A00A12F753600C2AF120EB27887E6FE760298
:10153A00120F337887EEF6E4F522F523F524F52524
:10154A00F526F565752C00752D00D2AF1205971298
:10155A000EB278A4E66006D293D295D29730740977
:10156A00C3E5369404400201CB41E6901A0D782077
:10157A001215F9E520B45A0CA31215F9E520B4A501
:10158A0003021597120EC71215B70215B6901A0361
:10159A0078807B0A1215F9A308DBF9901A0F788C68
:1015AA007B191215F9A308DBF9901A2822C2AF1287
:1015BA001638121612901A00740E1215FEA374062B
:1015CA001215FEA374151215FE901A0378807B0A71
:1015DA001215FDA308DBF9901A0F788C7B191215E6
:1015EA00FDA308DBF912164B121629901A2822E4D9
:1015FA0093F622E6438F01538FFD75EF0275B7A567
:10160A0075B7F1F0538FFE22438F02438F0175EFB6
:10161A000275B7A575B7F1901A0DF0538FFC229099
:10162A001A0D745AB1FE901A0E74A5B1FE227A30C0
:10163A0079D07820901A40B1F9E520F709A3DAF7B2
:10164A00227A3079D0901A40E7B1FE09A3DAF9225A
:10165A00AB74A875BB01027984BB02027985BB030E
:10166A00027986BB04027992BB05027987BB06021E
:10167A0079A3BB0702799CBB08027988BB09027966
:10168A0089E8F7227C0512059CDCFB22C2AF120511
:10169A00AC1205B31205BA1205C112058D1205ACBA
:1016AA001205B31205BA1205C112058D1205AC1244
:1016BA0005B31205BA1205C1D2AF22C2AF1205C1D3
:1016CA001205BA1205B31205AC12058D1205C11224
:1016DA0005BA1205B31205AC12058D1205C1120521
:1016EA00BA1205B31205ACD2AF22AE74AF75C2AF4F
:1016FA001205AC1205AC1205AC12058DDEF212050C
:10170A00C112058DDFF8D2AF22D196D18ED18E7556
:10171A007401757501757600D1F47C05AD5C12050E
:10172A009CC3ED955C70F5C3E55C9401400AC3E582
:10173A005C94FF403202174FD15AB1B7D196C2AF6B
:10174A0075EF12D18EDCD50576C3E5769403500287
:10175A0080C6D18E0575E5741490009F93F808C36E
:10176A00E57598500280AED18ED18E0574C3E574AA
:10177A00940A5002809C120EC7B1B7C2AF75EF121D
:02178A00D18EFE
:0319FD00021018BD
:101A00000E0615FFFFFFFF0304070101015AA501A0
:101A1000FFFFFFFFFF03FFFFFF25D0FAFA04FF01DE
:091A2000007AFF0101000300FF40
:101A4000235467794B4631323041485623202020B9
:101A500023424C48454C4923463331302320202033
:101A60002020202020202020202020202020202076
:101C0000C2AFC2D353D9BF7581C043B20343FF8073
:101C1000752438752503B1C975EF0275E24043F1AB
:101C20000853A4F775D4FFD2837DFA780379E67C54
:101C300010752200752300901DD67B0675249875BB
:101C400025013083028142208308D8FBD9F9DCF7D3
:101C500081B4308308D8FBD9F9DCF781B4B189E4C9
:101C600093A3C39A6004DDC381B4DBDBB17B600264
:101C7000812B7B08E493FAA3B15CDBF87A30B15C8A
:101C8000752200752300B17BEAFCEBFDC3ED94FEE9
:101C9000400EB17B8A278B28ED30E0048A828B834B
:101CA000B17B7AC270D8C3ED94FE601350CEBD00F4
:101CB00025EC60097520007521FF0200008100A855
:101CC00027A9280809D804D90281D3B17FEA89AAB3
:101CD000F281C50D81A0C3ED94035049EDA2E092BD
:101CE000007AC5C3E5829400E583941C50902000DF
:101CF00010438F02438F0175B7A575B7F1F030001F
:101D00001FA827A9280809438F01538FFDD804D99C
:101D100002A12089AAE275B7A575B7F1F0A3A10DBC
:101D2000538FFC817C7AC1BD030CE493A3FAB140CC
:101D3000DCF8B138817C817EAA22AB23B15CEBFA5E
:101D4000EA6222752608C3E52313F523E52213F57D
:101D50002250066323A0632201D526EAB1C9B1C986
:101D600075260AEAF4200102D283300102C283B14F
:101D7000C9C3134002C201D526EB22B17FEAFB2082
:101D80008302A17F308302A184752608AE24AF258B
:101D9000C3EF13FFEE13FEB1CDB1C9C3EA13308315
:101DA000024480FA30E703632201C3E52313F523DD
:101DB000E52213F52250066323A0632201D526D91C
:101DC000E52265236523F52222AE24AF250E0FDE22
:101DD000FEDFFCD20122424C48656C693437316326
:041DE000F3100601F5
:00000001FF
